:1000000012C02CC02BC02AC029C028C027C026C0BF
:1000100025C024C023C022C021C020C01FC01EC0D4
:100020001DC01CC01BC011241FBECFE5D4E0DEBF25
:10003000CDBF10E0A0E6B0E0EAE8F0E002C0059035
:100040000D92A036B107D9F710E0A0E6B0E001C0EC
:100050001D92A036B107E1F702D015C0D1CFBB9AEF
:1000600029E130E0C39A80E197E2F9013197F1F795
:100070000197D9F7C39880E49CE9F9013197F1F72A
:0A0080000197D9F7EFCFF894FFCFF6
:00000001FF
